:100315000178FF017900413C5500017A03413C56C3
:0C03250000413C5703017B00413C5D009F
:1010260012109FE4F53DE53D60031243E8123A22B3
:10103600AF631263E9124AC2E4F53DE53D6003126F
:1010460053B1AF71EF14601114601314601514607E
:101056001714601980007571011201C080121260A8
:10106600FE800D12601980081247848003125627ED
:10107600AF631263E9124AC290AC0074FFF090A805
:1010860000F012618AE4F53DE53DC3940850B3AF24
:091096003D1269DF053D80F022E6
:030023000257364B
:03003B00021B4065
:10017000120100010000004063073310210200005B
:10018000000109023500010100A005090400000575
:10019000FF000000070582034000010705840220DC
:1001A000000007050202400000070586022000004B
:0D01B00007050402200000040309040000FC
:10033100C103017100014310014610014A10014E31
:1003410010015110015510015910015E1001630097
:10035100018C000180000164FF018A00018B000112
:0B0361003500013600013700013800B4
:05036C00C10E017C0040
:10010000202A2A2A204D6964696D616E2055534268
:10011000204D69646953706F727420387838202AD2
:100120002A2A204669726D776172652052656C6576
:1001300061736520322E3231202A2A2A20436F70C3
:100140007972696768742028632920323030302D35
:1001500032303032204D6964696D616E20496E63C2
:060160002E202A2A2A20AD
:09037100019300019400019500C4
:10037A00413C60FFC109C10A01767F01747FC1084F
:09038A0001757F01770101730088
:08039300018D00038EFF66A43A
:03039B00017E00E0
:03000B000269ED9A
:10039E000196FF010B00010C7D010DC00111000142
:0903AE00127C0113C0413C610006
:1001C00090A00074EFF012618AE4F570C200C207DB
:1001D000C206C20F753962E539600AE571B40105DE
:1001E0001269C180F2C20230020302028CE571641E
:1001F00001600302028C907FD6E054F7F07539F469
:1002000020020EE539600AE571B401051269C1806A
:10021000EF7539F420020EE539600AE571B4010585
:100220001269C180EF7539F420020EE539600AE5E4
:1002300071B401051269C180EF7539F420020EE531
:1002400039600AE571B401051269C180EF7539F4AE
:1002500020020EE539600AE571B401051269C1801A
:10026000EF200283E571640160030201E7907FD60D
:10027000E04408F075390CE53970030201E7E571D7
:10028000640160030201E71269C180EBE57164015A
:10029000706D200F6A30020FC2021241DE907FAEF5
:1002A000E04402F075700212095D120BD0120E2CA0
:1002B000125505789606E6B40700501C9002C3F864
:1002C0002828730202DC0202E10202E60202EB02CB
:1002D00002F00202F50202FAE47896F61245BC80BA
:1002E000AB1207D080A612682A80A11266C3809C38
:1002F0001248C080971229378092126841808D90F1
:0E0300007FAEE054FDF0907FD6E04408F0227E
:10095D00907FB8E030E103020BCF907FE3747EF01F
:10096D00E4907FE4F0F516123F668F15EFD39400F7
:10097D00402A0516533B7F752304E515B4031D125C
:10098D003F668F15EFD3940040120516E515B4039D
:10099D000B123F66EFD3940040020516123FB58F40
:1009AD0015EFD39400402A0516533BBF752404E57B
:1009BD0015B4031D123FB58F15EFD39400401205EA
:1009CD0016E515B4030B123FB5EFD39400400205A5
:1009DD00161240048F15EFD39400402A0516533B91
:1009ED00DF752604E515B4031D1240048F15EFD3F2
:1009FD00940040120516E515B4030B124004EFD315
:100A0D009400400205161240538F15EFD394004009
:100A1D002A0516533BEF752804E515B4031D124046
:100A2D00538F15EFD3940040120516E515B4030B43
:100A3D00124053EFD394004002051612418F8F15CB
:100A4D00EFD39400402A0516533BFE753104E5158E
:100A5D00B4031D12418F8F15EFD39400401205166C
:100A6D00E515B4030B12418FEFD394004002051628
:100A7D00E51664107003020BC31240A28F15EFD35D
:100A8D00940040390516533BF7752A04E5156403A8
:100A9D00702BE516C3941050241240A28F15EFD37E
:100AAD00940040190516E515B40312E516C394100C
:100ABD00500B1240A2EFD3940040020516E51664C8
:100ACD00107003020BC31240F18F15EFD394004049
:100ADD00390516533BFB752C04E5156403702BE5A6
:100AED0016C3941050241240F18F15EFD39400408B
:100AFD00190516E515B40312E516C39410500B1223
:100B0D0040F1EFD3940040020516E5166410700312
:100B1D00020BC31241408F15EFD3940040390516D7
:100B2D00533BFD752E04E5156403702BE516C39438
:100B3D001050241241408F15EFD394004019051623
:100B4D00E515B40312E516C39410500B124140EF96
:100B5D00D3940040020516E516C394105058798AB7
:100B6D00E7788B66605005161269A1907FE5EFF06E
:100B7D00751501798AE7788B66601C1269A1907FE3
:100B8D00E5EFF00515798AE7788B66600A1269A1A1
:100B9D00907FE5EFF00515E51524FE600C14600E51
:100BAD0024027012E4907FE5F0E4907FE5F0E51506
:100BBD002480907FE5F0E516600825E025E0907F24
:030BCD00B9F0225A
:100BD000E50B14602414603E146075240360030266
:100BE0000E2B907FC8E030E103020E2B907FC9E00E
:100BF000FF1313543FF50A050BE50A7017F50B9028
:100C00007FC9F07A7D79C07E7D7FC0747DF50C74DC
:100C1000C0F50D22050B907FE3E50CF0E50D2403F4
:100C2000907FE4F0907FE5E0F509540FF508701728
:100C3000F50B907FC9F07A7D79C07E7D7FC0747D91
:100C4000F50C74C0F50D22E509C4540FF509050B28
:100C5000E509602A24FE7003020CD924FE70030209
:100C60000D3424FE7003020D8F24FE7003020DEA82
:100C700080007404250DF50D150A750B0122E50899
:100C8000D39543400D908005E020E503020E2B75BF
:100C90004310907FE3E50CF0907FE4E50DF0E5086C
:100CA00014601A14600D147024907FE5E0908000A9
:100CB000F01543907FE5E0908000F01543907FE5CC
:100CC000E0908000F01543533C7F752504740425A3
:100CD0000DF50D150A750B0122E508D3954A400D57
:100CE000908805E020E503020E2B754A10907FE303
:100CF000E50CF0907FE4E50DF0E50814601A14604F
:100D00000D147024907FE5E0908800F0154A907FE4
:100D1000E5E0908800F0154A907FE5E0908800F0CB
:100D2000154A533CDF7529047404250DF50D150A89
:100D3000750B0122E508D39551400D909005E020F8
:100D4000E503020E2B755110907FE3E50CF0907FC8
:100D5000E4E50DF0E50814601A14600D1470249099
:100D60007FE5E0909000F01551907FE5E0909000D5
:100D7000F01551907FE5E0909000F01551533CF74D
:100D8000752D047404250DF50D150A750B0122E56A
:100D900008D39559400D909805E020E503020E2BED
:100DA000755910907FE3E50CF0907FE4E50DF0E5D8
:100DB0000814601A14600D147024907FE5E0909878
:100DC00000F01559907FE5E0909800F01559907F5C
:100DD000E5E0909800F01559533CFD753204740419
:100DE000250DF50D150A750B0122E508D395645004
:100DF0003A907FE3E50CF0907FE4E50DF0E5081410
:100E0000601614600B147018907FE5E0FF12620A00
:100E1000907FE5E0FF12620A907FE5E0FF12620A30
:0C0E20007404250DF50D150A750B012258
:100E2C00E51114602414603414606124036003021F
:100E3C001025907FCCE030E103021025907FCDE0AF
:100E4C00FF1313543FF5100511E510700DF51190BB
:100E5C007FCDF075127C7513C0220511907FE3E5F0
:100E6C0012F0E5132403907FE4F0907FE5E0F50F9A
:100E7C00540FF50E700DF511907FCDF075127C7539
:100E8C0013C022E50FC4540FF50F0511E50F1460C4
:100E9C002024FE607724FE7003020F7324FE70037F
:100EAC00020FCE800074042513F513151075110173
:100EBC0022E50ED39546400D908405E020E5030213
:100ECC001025754610907FE3E512F0907FE4E51352
:100EDC00F0E50E14601A14600D147024907FE5E098
:100EEC00908400F01546907FE5E0908400F0154664
:100EFC00907FE5E0908400F01546533CBF752704C5
:100F0C0074042513F513151075110122E50ED395F4
:100F1C004E400D908C05E020E503021025754E1017
:100F2C00907FE3E512F0907FE4E513F0E50E14609A
:100F3C001A14600D147024907FE5E0908C00F0156D
:100F4C004E907FE5E0908C00F0154E907FE5E090A0
:100F5C008C00F0154E533CEF752B0474042513F5DF
:100F6C0013151075110122E50ED39555400D909473
:100F7C0005E020E503021025755510907FE3E5127E
:100F8C00F0907FE4E513F0E50E14601A14600D1474
:100F9C007024907FE5E0909400F01555907FE5E08B
:100FAC00909400F01555907FE5E0909400F0155565
:100FBC00533CFB75300474042513F513151075118F
:100FCC000122E50ED3955E400A909C05E030E54980
:100FDC00755E10907FE3E512F0907FE4E513F0E589
:100FEC000E14601A14600D147024907FE5E0909C30
:100FFC0000F0155E907FE5E0909C00F0155E907F10
:10100C00E5E0909C00F0155E533CFE7533047404CF
:0A101C002513F513151075110122BC
:10078B00907FDE7404F0907FDF7414F0907FDD7443
:0C079B0018F0E4907FC9F0907FCDF022B0
:1007D000AF70EF146019146037800090A00074EFC0
:1007E000F0757001126A24EF2451903C61F02212DE
:1007F0006A24903C61E06F704790A000E06410F0C4
:10080000126A24EF2451903C61F07889E6F51422B5
:10081000126A24903C61E06F7026126A24EF245122
:10082000903C61F07889E6FFB51413907FAEE054F8
:10083000FDF090A00074EFF0757001D20F228F14BC
:010840002295
:08075C00907FB4E04402F0229A
:0907C500907FAFE04408F0D3225C
:0207CE00D32234
:0300330002075869
:0407580053D8EF3251
:02095300D322AD
:09094100907FEAE07898F6D322D9
:0F0923007898E6907F00F0907FB57401F0D322B2
:09094A00907FEAE07897F6D322D1
:0F0932007897E6907F00F0907FB57401F0D322A4
:02095500D322AB
:02095700D322A9
:02095900D322A7
:02095B00D322A5
:0B03B700017F01019901C190019A0330
:1005D900C0E0C083C082C085C084C086758600C063
:1005E900D075D000C000C006C0075391EF907FAB13
:1005F9007402F0788906301018157FE57F70359000
:10060900A00074FFF0C210C3741E789A96F57F801B
:1006190023D57F2090A00074EFF0D2107899E6FFDF
:100629000826F6FE64036004EEB41D06EFF40478B0
:1006390099F68E7FD007D006D000D0D0D086D0844E
:09064900D085D082D083D0E032CC
:010562003266
:10076400C0E0C083C082C085C084C086758600D2C4
:10077400025391EF907FAB7401F0D086D084D08582
:07078400D082D083D0E032E7
:10058D00C0E0C083C082C085C084C086758600D29D
:10059D00075391EF907FAB7408F0D086D084D0854F
:0705AD00D082D083D0E032C0
:10056300C0E0C083C082C085C084C0867586009009
:100573007FC4E4F05391EF907FAB7404F0D086D046
:0A05830084D085D082D083D0E0320E
:1005B400C0E0C083C082C085C084C08675860053F5
:1005C40091EF907FAB7410F0D086D084D085D08228
:0505D400D083D0E032ED
:010657003270
:01065B00326C
:010652003275
:010653003274
:010654003273
:010655003272
:010656003271
:01065800326F
:01065900326E
:01065A00326D
:01065C00326B
:01065D00326A
:01065E003269
:01065F003268
:010660003267
:010661003266
:03004300020700B1
:10070000020764000205D9000205630002058D009E
:100710000205B40002056200020652000206530000
:100720000206540002065500020656000206570053
:10073000020658000206590002065A0002065B0033
:1007400002065C0002065D0002065E0002065F0013
:080750000206600002066100D0
:10109F00538EF8907F96E04480F0E04440F0907FCC
:1010AF0093740CF0907F9C74FCF0907F947401F01B
:1010BF00907F9D74FAF0907F9574C0F0907F9E742E
:1010CF00F2F0907F94E0440CF0907F9DE054FBF0A1
:1010DF00E04408F0907F95E04403F0907F9EE05449
:1010EF00FEF0E04402F075B850907F92E04402F0B9
:1010FF005389F0E4F58CF58AD28CD2A9126A1DD2ED
:10110F00AFE589540F2420F589758DFE758BFED2BE
:10111F008EC2AC759850C298C299C2AE75C050C2FB
:10112F00C0C2C1D2AE907FD6E04408F0E04404F0D4
:10113F00E04402F012078BC2E853D8DF907FAE7401
:10114F001DF0907FAB74FFF0907FA9F0907FAAF015
:10115F005391EF907FAF7401F0C202D2E843D820D1
:10116F001260B4753BFF753CFFE47889F6D204D268
:10117F0005F525F523F527F524F529F526F52BF5A6
:10118F0028F52DF52AF530F52CF532F52EF533F53A
:05119F003112618A22FB
:1008F200907FD6E030E712E04401F07F147E0012D0
:0A090200090C907FD6E054FEF022AD
:1008D100907FD6E04480F0438701000000000022B1
:020890008F18BF
:10089200E4F519751AFF751B01751CB7AB1AAA1B73
:1008A200A91C90000112048AB4031DAF190519EFA7
:1008B200B51801221204717E0029FFEE3AA90775CC
:0E08C2001AFFF51B891C80D47B007A00790098
:0108D0002205
:10084100E4FE751AFF751B01751C82AB1AAA1BA960
:100851001C90000112048A6402702DAD060EEDB5E4
:100861000701229000021204B785F018F5196218E9
:10087100E5186219E519621829FDE5183AA9057507
:0E0881001AFFF51B891C80C37B007A007900EA
:01088F002246
:10090C008E158F16E5161516AE15700215154E6060
:07091C00051208E180EE2244
:1008E1007400F58690FDA57C05A3E582458370F92A
:0108F10022E4
:030000000203C335
:0C03C300787FE4F6D8FD75819A02040AE8
:10044F00C2D530F707B2D563F0FF05F030E70CB235
:10045F00D5F4048463F0FF05F080018430D502F4F5
:02046F00042265
:10047100BB010689828A83E0225002E722BBFE0289
:09048100E32289828A83E49322BC
:10048A00BB010CE58229F582E5833AF583E0225027
:10049A0006E92582F8E622BBFE06E92582F8E22271
:0D04AA00E58229F582E5833AF583E493228B
:1004B700BB0110E58229F582E5833AF583E0F5F083
:1004C700A3E0225009E92582F886F008E622BBFE60
:1004D7000AE92582F8E2F5F008E222E5832AF583A6
:0804E700E993F5F0A3E993226B
:0604EF008A838982E47398
:1003CF00021026E493A3F8E493A34003F68001F20E
:1003DF0008DFF48029E493A3F85407240CC8C3332F
:1003EF00C4540F4420C8834004F456800146F6DFFE
:1003FF00E4800B0102040810204080900315E47E76
:10040F00019360BCA3FF543F30E509541FFEE493F2
:10041F00A360010ECF54C025E060A840B8E493A3B9
:10042F00FAE493A3F8E493A3C8C582C8CAC583CAE4
:10043F00F0A3C8C582C8CAC583CADFE9DEE780BE9C
:0103C200003A
:00000001FF
